:020000020000FC
:1000000002C06CC06CC03FED3DBF37E137BBC09A4A
:10001000C19AC29A00E010E020E0C1981A94F1F76A
:100020002A94E1F7C19A31E033BF32E039BF7894C6
:10003000AA271ED0660F35E0A60F3A95E9F718D02B
:10004000A60FA03210F03FE1A32F19D0623711F0B4
:10005000623511F40A2FECCF673611F0673411F4D2
:100060001A2FE6CF623611F0623409F42A2FE0CF5E
:1000700006D06033E8F36A33D8F76053089549E057
:10008000B399FECFF8947DE20FD07AE50DD0889435
:10009000C49AB3990894C4984A9511F06795F5CF1E
:1000A000332732BF78940895332732BF04D082B704
:1000B0008717E8F308950FB6903221F49927C09876
:1000C000C198C298901708F0C09A911708F0C19A89
:1000D000921708F0C29A93950FBE08951895EBDF1A
:0200E000189571
:00000001FF
